:020000040000FA
:10300000E4EF19F0EAEF19F0EBEF19F0ECEF19F03B
:10301000EDEF19F005EF1AF04DEF1AF04EEF1AF040
:103020004BEF1AF04CEF1AF04FEF1AF048EF1AF08E
:1030300047EF1AF036EF1AF046EF1AF080EF19F06A
:1030400081EF19F082EF19F083EF19F04AEF1AF0CF
:1030500049EF1AF0120000001200000012000000F8
:103060001200000012000000120000001200000018
:103070001200000012000000120000001200000008
:10308000FFFFFFFFFFFFFFFFFFFFFFFFFFFFFFFF50
:10309000FFFFFFFFFFFFFFFFFFFFFFFFFFFFFFFF40
:103300001200120012001200036A046A88EF19F01A
:103310008C9A8C9C04B08C8C8C8A8C9A8C9C04B279
:103320008C8C8C8A8C9A8C9C04B48C8C8C8A8C9A15
:103330008C9C04B68C8C8C8A8C9A8C9C04B88C8C5B
:103340008C8A8C9A8C9C04BA8C8C8C8A8C9A8C9CDF
:1033500004BC8C8C8C8A8C9A8C9C04BE8C8C8C8A41
:103360008C9A8C9C03B08C8C8C8A8C9A8C9C03B22B
:103370008C8C8C8A8C9A8C9C03B48C8C8C8A8C9AC6
:103380008C9C03B68C8C8C8A8C9A8C9C03B88C8C0D
:103390008C8A8C9A8C9C03BA8C8C8C8A8C9A8C9C90
:1033A00003BC8C8C8C8A8C9A8C9C03BE8C8C8C8AF3
:1033B0008C9A8B888C9C8B988B9A030E056A052AB5
:1033C0000562FDD78B8A120084EC19F0116A50EC6B
:1033D0001AF0120012001200120082EC16F0F20E27
:1033E000F66E330EF76E9EEC16F09EEC16F0108023
:1033F0001200000F5465737420534944204D6F64CC
:10340000756C6500400450696E3A10A0120010906F
:10341000450E88EC16F0300EF66E340EF76E115035
:10342000040DF350F626F450F722040E9CEF16F02C
:1034300041302020413120204132202041332020C2
:103440004134202052455323443020204431202051
:10345000443220204433202044342020443520208E
:103460004436202044372020435323200350F00BC0
:10347000B00A0BE10450010A08E10550116E0F0E6D
:103480001160116A108050EC1AF012001200120044
:10349000120012001200120012001200120012009C
:1034A0008B9A036A046A1150F10FD8B0F10E0F0F16
:1034B000C8EC16F00ED011D014D017D01AD01DD0F1
:1034C00020D023D026D029D02CD02FD032D035D028
:1034D00038D0010E036E88EF19F0020E036E88EFEC
:1034E00019F0040E036E88EF19F0080E036E88EFD2
:1034F00019F0100E036E88EF19F0200E036E88EF9E
:1035000019F0010E046E88EF19F0020E046E88EFB8
:1035100019F0040E046E88EF19F0080E046E88EF9F
:1035200019F0100E046E88EF19F0200E046E88EF6B
:1035300019F0400E046E88EF19F0800E046E88EFCB
:0635400019F08B9A120045
:00000001FF
